:020000040000FA
:0608000040EF16F01200AB
:020806001200DE
:06080800E2EF0DF012000A
:02080E00C250D6
:08081000020B01E0010E1200D1
:060818004AEF18F0120087
:02081E000700D1
:100820001C540000EE0700000500000019540000F1
:100830006C02000003000000DD530000B20700005E
:100840003C000000D95300006502000004000000D5
:10085000CC530000580200000D000000BA53000005
:100860002A02000012000000B853000073020000CA
:040870000200000082
:0C08740076EC09F0FB0EDBCFF3FFDB0697
:10088000F35000090AE0C4EC09F0FA0E2FEC0AF06C
:10089000F3E12C1CF1E1010E01D0000EA5EF09F0EF
:1008A00076EC09F03B0EE12402E3E168E652E16EEA
:1008B000010EDB6A020EDB6AF90EDBCFF6FFFA0EE1
:1008C000DBCFF7FFFB0EDBCFF8FF0800F550DF6E44
:1008D000DF5002E1CBEF08F0250EDF5C02E0BEEF57
:1008E00008F0030EDB6A040EDB6A050EDB6A060EF7
:1008F000DB6A070EDB6ADEEC08F02D0EDF5C0CE035
:100900002B0EDF5C09E0200EDF5C06E0230EDF5CCF
:1009100003E0300EDF5C1AE1DF50300A14E0130A06
:100920000FE0030A0AE00B0A05E0060AE4E1030E01
:10093000DB80E1D7030EDB82DED7030EDB84DBD75F
:10094000030EDB86D8D7030EDB88D5D72A0EDF5CF3
:100950001BE1DAEC08F028EC09F010E0030EDB8074
:100960001D681E68130EDBCF22F0140EDBCF23F0C0
:100970008EEC26F0040E1BC0DBFF03D0130E11EC2F
:1009800009F0DEEC08F00BD0090EDB6A7FEC09F011
:1009900003E0F3EC09F0FAD7090E11EC09F0030EAD
:1009A000DBB0DB982E0EDF5C1BE1DEEC08F02A0EDC
:1009B000DF5C0BE1DAEC08F028EC09F003E1130E40
:1009C00063EC09F0DEEC08F00BD0090EDB6A7FEC7B
:1009D00009F003E0F3EC09F0FAD7090E63EC09F033
:1009E000680EDF5C07E1DEEC08F0680EDF5C1DE1FD
:1009F000030E18D0740EDF5C17E07A0EDF5C14E093
:100A0000480EDF5C06E0540EDF5C03E05A0EDF5C4C
:100A100002E1020E07D06C0EDF5C03E06A0EDF5CC1
:100A200004E1010EB6EC09F0C9DBDF506E0A01E10A
:100A300081D31E0A01E192D1200A01E18FD13F0A40
:100A400001E149D11A0A01E146D10D0A01E143D180
:100A5000200A01E140D13A0A01E13DD1200A01E139
:100A60003AD1260A01E135D10D0A01E132D11A0A43
:100A700001E1D9D0200A4AE0300A1FE0460A0EE020
:100A8000250A01E085D3D950F90FE96EFF0EDA206F
:100A9000EA6E010EEE5E000EEE5AEE5AC4EC09F05C
:100AA000250EE66E95DB03E12C1C01E16BD3C0EC57
:100AB00009F001E26DD3DB2A6BD3080EDB6A040E6A
:100AC000DB50010806E2040EDB0488EC09F0DB5081
:100AD0008BDB080EDB5009E0030EDB50010B05E158
:100AE00072DB01E04FD3080EDB6A64DBEFCFDFFF80
:100AF00038EC0AF003E12C1C01E144D3C0EC09F00E
:100B000001E3DB2A60DB01E143D33CD3070EDB507A
:100B100002080FE104EC0AF0030ECBEC09F00E0E14
:100B2000EECFDBFF0F0EEECFDBFF100EEECFDBFFC5
:100B300020D0F70EDBCF2EF0F80EDBCF2FF0020E19
:100B40002E5E000E2F5AF70E2EC0DBFFF80E2FC0C0
:100B5000DBFF2EC0E9FF2FC0EAFFBBEC09F02D6AD6
:100B60000E0E2BC0DBFF0F0E2CC0DBFF100E2DC0B6
:100B7000DBFF0E0EDBCFE6FF0F0EDBCFE6FF100E26
:100B8000DBCFE6FF4BEC26F0E552E552E552130EC3
:100B90001CC0DBFF140E1DC0DBFF060EDB5005E0A2
:100BA000130EFFEC09F001E26ADB23EC0AF002E22B
:100BB000130E37DBE6EC09F006E0040EFFEC09F05B
:100BC00002E2050E2EDB030EDBB005D0FCDA01E0FD
:100BD000D9D2080EDB6A090EDB6A0E0EDBCFF6FFF8
:100BE0000F0EDBCFF7FF100EDBCFF8FF0800F5503C
:100BF000DF6EDF5014E029EC0AF011E238EC0AF065
:100C000003E12C1C01E1BED2BBDB01E3DB2A090EB0
:100C1000DB2AD9500E0FE96E000ECBDBE7D7D3DA13
:100C200001E1B6D2AFD2C6DA110EEECFDBFF120E63
:100C3000EDCFDBFF110EDBCFE6FF120EDBCFE6FFC1
:100C40003DEC26F0E552E552130EF3CFDBFF140E18
:100C5000F4CFDBFF060EDB5004E0130ED0DB01E225
:100C60000EDB23EC0AF002E2130EDBDAAFDB05E069
:100C7000040EC5DB02E2050ED4DA030EDBB005D0AC
:100C8000A2DA01E07FD2080EDB6A090EDB6A110EE0
:100C9000DBCFE9FF120EDBCFEAFFEFCFDFFFDF5044
:100CA00014E0D7DB12E2E4DB03E12C1C01E16AD2A1
:100CB00067DB01E3DB2A090EDB2A110EDB2ADBCF1F
:100CC000E9FF120EE8E3DB2AE6D77DDA01E160D224
:100CD00059D2030EDB8E070EDB0410E195DB040E08
:100CE0005ADB0A0EEECFDBFF0B0EEECFDBFF0C0E56
:100CF000EECFDBFF0D0EEECFDBFF6CD0070EDB502F
:100D000003082CE1030EDBAE0DD0B2DA020E76DA68
:100D1000EFCF2BF02C6A2D6A2E6A2BAE39D02C68BF
:100D20002D6835D0F70EDBCF2CF0F80EDBCF2DF091
:100D3000020E2C5E000E2D5AF70E2CC0DBFFF80EB3
:100D40002DC0DBFF2CC0E9FF2DC0EAFFEFCF2BF059
:100D50000A0E2BC0DBFF0B0EDB6A38D0070EDB5010
:100D6000020809E1030EDBAE04D059DB2DAE10D032
:100D70000ED055DB0DD0030EDBAE12D079DA020EA9
:100D80003DDAF9DA2D6A2E6A2CAE02D02D682E6873
:100D9000E2DA0C0E2DC0DBFF0D0E2EC0DBFF1AD0E9
:100DA000F70EDBCF2DF0F80EDBCF2EF0020E2D5E0E
:100DB000000E2E5AF70E2DC0DBFFF80E2EC0DBFF03
:100DC0002DC0E9FF2EC0EAFFD6DAC5DA0C0EDB6AC9
:100DD0000D0EDB6A060EDB5005E1010EF36E050E0B
:100DE000F3CFDBFF150EDB6A160EDB6AD950370F27
:100DF0002B6E000EDA202C6E390E2BC0DBFF3A0E64
:100E00002CC0DBFF380EDB6A080EDB6A0A0EAEDA96
:100E1000DF50780A12E0200A10E0280A0CE0200ACD
:100E20000AE03F0A06E00D0A02E0200A08E1020E8D
:100E300005D0080E03D0080EDF26100E97DA030E39
:100E4000DBBE02D0DB92DB94DB50800B26E08ADA3B
:100E5000030EEB50000AE8AE02D0D89008D0000E86
:100E6000EE5C000EEE58000EEE58000EEE5815E245
:100E700011DA206821682268236889EC27F00A0EBD
:100E800017C0DBFF0B0E18C0DBFF0C0E19C0DBFF19
:100E90000D0E1AC0DBFF2D0E08D0030EDBA202D010
:100EA0002B0E03D0DBA408D0200EF36E170EF3CF69
:100EB000DBFF150EDB2A02D0170EDB6A050EDB50B6
:100EC00003E1B5D901E189D0740E2B6E530E2C6E5F
:100ED000000E2D6E070EDBCF2EF02F6A306A316ABE
:100EE0002EC020F02FC021F030C022F031C023F0FE
:100EF000D1D9E5EC28F02B501724F36E2C50182094
:100F0000F46E2D501920F86EF4CFF7FFF3CFF6FFF3
:100F10000800090EF5CFDBFF580EDF5C0FE1610E14
:100F2000F36E090E79D90AE3200E2B6E090EDBCF82
:100F3000E7FF2B50E75E090EE7CFDBFF070EDBCFA5
:100F40002BF02C6A2D6A2E6A0DDA2BC020F02CC0F3
:100F500021F02DC022F02EC023F0EECF1BF0EECFFB
:100F60001CF0EECF1DF0EFCF1EF0E5EC28F01EC018
:100F7000EDFF1DC0EDFF1CC0EDFF1BC0EFFF390EE4
:100F8000DBCFE9FFDB063A0EDBCFEAFF01E2DB064F
:100F9000090EDBCFEFFF150EDB2A49D995E1030ED1
:100FA000DBA61DD06F0EDF5C06E1BFD918E3150E7E
:100FB000DB2859DA14D0780EDF5C09E0580EDF5CCC
:100FC00006E0620EDF5C03E0420EDF5C08E1020E29
:100FD000F36E160EF3CFDBFF02D0150EDB6A030EA5
:100FE000DB50100B0EE0040EDBCF2BF0050EDB50B8
:100FF000D8802B5406E2060EDB5003E1040EDB50D2
:1010000032DA93D90AE2050EDBCFE7FF150EDB508B
:10101000E75E050EE7CFDBFF02D0050EDB6A040EAC
:10102000DBCF2BF0160E43D9D8802B5414E2160ECA
:10103000DBCFE6FF150EDBCFE6FF040EDBCFE6FFCE
:10104000050EDB50E552E75CE552D880E754E552E7
:10105000D880E7545DD9030EDB50010B0BE1080E7D
:10106000DB5008E0B0D801E08DD0080EDB50BCD8D2
:10107000080EDB6A170EDB5007E086D9170EEFD992
:1010800003E12C1C01E17ED0160EDB5016E07CD96A
:10109000300EE66E9DD802E12C1C74E075D9DFCFCE
:1010A000E6FF05EC27F0E552E552E552F4CF2CF0CF
:1010B0000001F31C02E12C1C65E0050EDBCF2BF0D8
:1010C000160EDB50D8802B5409E2050EDBCFE7FF6C
:1010D000160EDB50E75E050EE7CFDBFF300EE66E47
:1010E000050EC9D94FE1390EDB2ADBCFE9FF3A0EF5
:1010F00001E3DB2ADBCFEAFF090EEFCFDBFFDB509A
:101100000EE042D9090EABD902E12C1C3BE0390EAE
:10111000DB2ADBCFE9FF3A0EEDE3DB2AEBD753D82E
:1011200031E1160EDBCFE6FF080EC1D8E552E72409
:101130005BD82ED0070EDB50030A1CE0010A14E036
:10114000030A07E079D9DBCFEEFF020EDBCFEDFF1C
:101150001FD0F3D8306A2EAE02D02F6830682AD85C
:10116000BAD830C0EEFF14D0E8D82EBE2F6822D8EF
:10117000B2D80ED061D9DBCFEFFF0AD079D905E123
:101180002C1C03E1F368F46810D0FAD801E3DB2AE1
:1011900077D965EF04F0010EDBCF2BF0020EDBCF29
:1011A0002CF02BC0F3FF2CC0F4FFD9CFE1FFDACF36
:1011B000E2FFCBD029D9020ECBEF09F061D90800AC
:1011C000F550DF6E1200200EE66E080E3BEF0AF0BF
:1011D00005EC27F0E552E552E552F3CF2BF0F4CFC2
:1011E0002CF00001F31C12002B6E2C6AD950010F59
:1011F0004DD92B50EE262C50ED2212002F5E000E02
:10120000305AF70E2FC0DBFFF80E30C0DBFF2FC0C7
:10121000E9FF30C0EAFF1200DBCFF4FFF350F45CCB
:101220001200DB50E76E040EE7CFDBFF12000A0E60
:10123000DBCF2BF00B0EDBCF2CF00C0EDBCF2DF029
:101240000D0EDBCF2EF02B502C102D102E10120077
:10125000130EEECFDBFF140EEDCFDBFF130EDBCF53
:101260002BF0140EDBCF2CF00001800E2C1412009A
:10127000F70EDBCF2FF0F80EDBCF30F01200050EAB
:10128000DB50E66ED950130F01D9E552E750EE6EF0
:10129000ED6A12000A0EDBCF1BF00B0EDBCF1CF049
:1012A0000C0EDBCF1DF00D0EDBCF1EF01200DBCFDE
:1012B000E6FF150EDBCFE6FF050EDB50E552E72417
:1012C000E552E7241200DB50CED8010EF36E060E75
:1012D000F3CFDBFF1200EE50EFCFEAFFE96E2DC037
:1012E000EEFF2EC0EEFF2FC0EEFF1200D9CFE6FFBB
:1012F000DACFE6FFE1CFD9FFE2CFDAFF1200DFCF8E
:10130000E6FFE66A7FEC29F0E552E552F350120061
:10131000E76E080EE7CFDBFF1200EECF2BF0EECF2B
:101320002CF0EFCF2DF02E6A1200050EDBCF2BF044
:10133000150EDB50D8802B541200010EDBCF2DF0A0
:10134000020EDBCF2EF02F6A1200E552E5CFDAFF56
:10135000E7CFD9FF12000A0E2BC0DBFF0B0E2CC00B
:10136000DBFF1200D9500A0F46EF0AF0F36E070EAA
:10137000F3CFDBFF1200EECF2BF0EFCF2CF01200FB
:10138000010EDB2A020E1200FC0EDBCFE6FFFD0E83
:10139000DBCFE6FF12002B5E000E2C5AF70E2BC09F
:1013A000DBFFF80E2CC0DBFF2BC0E9FF2CC0EAFFEF
:1013B0001200DA20EA6EEF2AEECFF6FF000EEF22DF
:1013C000EECFF7FFEF22EECFF8FF1200040EDBCFD7
:1013D000E6FF130EDB50E552E75C9ADFDB5004DFDB
:1013E000060EDB501200090EDB500A0DF350DF240D
:1013F000D00FE76E090EE7CFDBFFDEEF08F0DB5022
:10140000F36E050E0CEF09F0F70EDBCF2BF0F80EA4
:10141000DBCF2CF01200DFCFE6FFE8EF08F028DF8B
:10142000030EECDE8DEF09F03AEC04F0E552E552E4
:10143000E552E55200091200BDDEEE50EFCFEAFFA3
:10144000E96E010E1200130EDB50F36E040E0CEF6A
:1014500009F0040EDB50F36E090E0CEF09F0DBCF40
:10146000E6FFE8EF08F0E76E050EE7CFDBFF1200BE
:101470008BDF0BEF0AF0DBCFE6FF86DF14EF0AF01D
:10148000D950F90FE96EFF0ED9EF09F0E96E000EA1
:06149000DA20EA6E1200F2
:0A149600E50EE66E09EC29F0E552C0
:1014A000F60ECF6E3B0ECE6E9F90120068DB0C0ED8
:1014B000E126F2AC04D0F29C24DBF28C01D021DBDB
:1014C000DECF2BF0DDCF2CF03B0E2B5EF60E2C5A30
:1014D0000A0E2BC0DBFF0B0E2CC0DBFF020EDBCF96
:1014E0002BF0030EDBCF2CF0040EDBCF2DF0050E1E
:1014F000DBCF2EF049DB89EC27F017C02BF018C0AA
:101500002CF019C02DF01AC02EF0020E1D6E1E6AAE
:101510000A0EDBCF22F00B0EDBCF23F070EC26F0AF
:101520001BC02FF01CC030F0050E226E236A1BC0BA
:101530001DF01CC01EF069EC29F0316A326A1D50A2
:101540002B261E502C2231502D2232502E22060ED8
:101550002BC0DBFF070E2CC0DBFF080E2DC0DBFF0E
:10156000090E2EC0DBFF060EDBCF2BF0070EDBCF04
:101570002CF0080EDBCF2DF0090EDBCF2EF019DB9F
:10158000D9CFE1FFF8D29FDADBDAD9CFE1FFF3D28E
:101590000ADBEECF2BF0EECF2CF0EECF2DF0EFCF1D
:1015A0002EF0A2D200DB0701B651EE5C2B6EB751D4
:1015B000EE582C6EB851EE582D6EB951EE582E6E75
:1015C00093D2D9CFE6FFD7D2DADA0701E251E3119D
:1015D0001CE1FB0EDBCF06F2FC0EDBCF07F2FD0EAB
:1015E000DBCF08F2FE0EDBCF09F206C202F207C221
:1015F00003F208C204F209C205F2F29CF90EDBCF35
:10160000E2F7FA0EDBCFE3F77BD0E451E5111CE102
:10161000FB0EDBCF0EF2FC0EDBCF0FF2FD0EDBCFAD
:1016200010F2FE0EDBCF11F20EC20AF20FC20BF265
:1016300010C20CF211C20DF2F29CF90EDBCFE4F7EE
:10164000FA0EDBCFE5F75CD0E651E7111CE1FB0EAB
:10165000DBCF16F2FC0EDBCF17F2FD0EDBCF18F25C
:10166000FE0EDBCF19F216C212F217C213F218C225
:1016700014F219C215F2F29CF90EDBCFE6F7FA0E5E
:10168000DBCFE7F73DD0E851E9111CE1FB0EDBCFE2
:101690001EF2FC0EDBCF1FF2FD0EDBCF20F2FE0EA2
:1016A000DBCF21F21EC21AF21FC21BF220C21CF2B3
:1016B00021C21DF2F29CF90EDBCFE8F7FA0EDBCF68
:1016C000E9F71ED0EA51EB111CE1FB0EDBCF26F24D
:1016D000FC0EDBCF27F2FD0EDBCF28F2FE0EDBCFB8
:1016E00029F226C222F227C223F228C224F229C2FA
:1016F00025F2F29CF90EDBCFEAF7FA0EDBCFEBF71F
:10170000F28C39D23CDAE2C72BF0E3C72CF02BDAAB
:1017100007E12DDA05E1F29C0701E26BE36B33D0C0
:10172000E4C72BF0E5C72CF01EDA07E120DA05E16B
:10173000F29C0701E46BE56B26D0E6C72BF0E7C708
:101740002CF011DA07E113DA05E1F29C0701E66BF0
:10175000E76B19D0E8C72BF0E9C72CF004DA07E1F2
:1017600006DA05E1F29C0701E86BE96B0CD0EAC7E9
:101770002BF0EBC72CF0F7D907E1F9D905E1F29C82
:101780000701EA6BEB6BF28CF6D1F29EF60ECF6E90
:101790003B0ECE6EF28E0701B22B000EB323B423A4
:1017A000B5230701BE510EE00701BA07000EBB5B6F
:1017B000BC5BBD5B0701BA51BB11BC11BD1102E19D
:1017C0000701BE6B0701DC5106E00701C32B000EC9
:1017D000C423C523C6230701DD5106E00701C72B3B
:1017E000000EC823C923CA230701DE5106E0070102
:1017F000CB2B000ECC23CD23CE230701DF5106E0F7
:101800000701CF2B000ED023D123D2230701E051B3
:1018100006E00701D32B000ED423D523D6230701DE
:10182000E15106E00701D72B000ED823D923DA2394
:101830000701E251E3111BE002010207000E035B06
:10184000045B055B020102510311041105110FE154
:1018500005D0E3C7FAFF0701E251F96EFADF06C2CD
:1018600002F207C203F208C204F209C205F207013C
:10187000E451E5111BE002010A07000E0B5B0C5B53
:101880000D5B02010A510B110C110D110FE105D076
:10189000E5C7FAFF0701E451F96EFADF0EC20AF25A
:1018A0000FC20BF210C20CF211C20DF20701E65189
:1018B000E7111BE002011207000E135B145B155BBE
:1018C000020112511311141115110FE105D0E7C7D0
:1018D000FAFF0701E651F96EFADF16C212F217C2DB
:1018E00013F218C214F219C215F20701E851E911F6
:1018F0001BE002011A07000E1B5B1C5B1D5B020153
:101900001A511B111C111D110FE105D0E9C7FAFF77
:101910000701E851F96EFADF1EC21AF21FC21BF26C
:1019200020C21CF221C21DF20701EA51EB111BE09B
:1019300002012207000E235B245B255B020122517A
:101940002311241125110FE105D0EBC7FAFF070180
:10195000EA51F96EFADF26C222F227C223F228C228
:1019600024F229C225F20701ED2B0701ED510A08E7
:1019700009E201010101E351010B04E004EC1DF057
:101980000701ED6B77EC14F0080E0101D515070186
:10199000EC5D09E00701EC5101E000D0080E010107
:1019A000D5150701EC6F02013E5123E0800E0101C5
:1019B000D5151FE15CEC1CF00201405D1AE0070147
:1019C000B651B711B811B91114E0FF0E0201405D14
:1019D00005E15CEC1CF00201406F0BD05CEC1CF0EC
:1019E0000201406F16EE00F026EE00F0010EFC6ED4
:1019F00010001200C4D8FB0EDBCF2BF0FC0EDBCFA7
:101A00002CF0FD0EDBCF2DF0FE0EDBCF2EF02B5099
:101A10002C102D102E1011E0FB0EDBCFBAF7FC0EB0
:101A2000DBCFBBF7FD0EDBCFBCF7FE0EDBCFBDF788
:101A30000701010EBE6FBE51FEE19DD0A0D8FE0E83
:101A4000DB5004E0FE0EDB50060804E2FE0EDB5025
:101A5000000E01D0010E8FD051D803E07CD8010ECA
:101A6000EF6E89D04BD802E076D8EF6A84D046D8A2
:101A70000EE059D8FA0EDBCFEEFFFB0EDBCFEEFF08
:101A8000FC0EDBCFEEFFFD0EDBCFEEFFF28C73D052
:101A900076D8040EE12680D805E11B6A1C6A1D6A0F
:101AA0001E6A0ED040D8EECFDFFF010EEECFDBFF77
:101AB000020EEECFDBFF030EEECFDBFFF28C40D841
:101AC000D9CFE1FF58D05BD8040EE126F29CB2C713
:101AD000DFFF010EB3C7DBFF020EB4C7DBFF030E4F
:101AE000B5C7DBFFF28C12004FD8E5EC28F01BC025
:101AF000F3FF1CC0F4FFD9CFE1FF3DD040D8CCEFBD
:101B00000DF0CE50DF6E010ECFCFDBFF020EB2C75D
:101B1000DBFF030EB3C7DBFF040EB4C7DBFF050E0C
:101B2000B5C7DBFF1200F29CFE0EDB50040DF3CFB5
:101B3000E9FFF4CFEAFFBF0EE926070EEA22120002
:101B4000DECF1BF0DECF1CF0DECF1DF0DDCF1EF0B0
:101B5000DD52DD521200FE0EDB50EA6ADB0FE96E49
:101B6000070EEA221200FD0EDB502B181200FE0EAB
:101B7000DB502C181200E552E7CFD9FF1200D9CF65
:101B8000E6FFE1CFD9FF1200E80E206E030E216EB2
:101B9000226A236AD9EF0DF0FE0EDBCFE6FF4EDF9F
:101BA000E552000912008FDFD9CFE9FFDACFEAFF53
:101BB00012002BC01BF02CC01CF02DC01DF02EC03D
:041BC0001EF0120001
:0C1BC400DACFE4FFE2CFDAFFE9CFE4FF64
:101BD000EACFE4FFE652F2A202D09CD802D09EB631
:101BE000C8D8E552E5CFEAFFE5CFE9FFE5CFDAFF58
:101BF0001100E66A010EE66E050EE66EC1EC27F0F6
:101C0000E552E552E5521200070EB46E000E886EE2
:101C1000876E866E856E846E836E826E816E806E38
:101C2000916E906E8F6E8E6E8D6E8C6E8B6E8A6ED8
:101C3000896E92689368BF0E946E956A700E966E68
:101C40009F0E976EE40E986E0F0E996E9A68C16E95
:101C5000070EC06EF19EB0989C8EA26A9F6AA06A21
:101C60009D6AA36AA56AC5DF9F86D08E9E969D86D3
:101C70009382F06AF288F09EF098F192F09AF16AFD
:101C8000F28CF28E1200D9CFE6FFE1CFD9FFE652F7
:101C9000BBDF0101E397E3990201A70E566F010E26
:101CA000576FDF6A100EDF5C0AE2DF50EA6A5625E2
:101CB000E96E5751EA227F0EEF6EDF2AF3D701015A
:101CC000C06B010EC16FC90EC26F0101E385010E29
:101CD000D56E800ED76EF90ED66ED59EA30EE66E2B
:101CE000010EE66E94D8E552E5520101E393A30E8E
:101CF000E66E010EE66E8BD8E552E5520101E393E4
:101D0000E552E552E7CFD9FF120082828088949293
:101D100092981200F2920201200E526F9F860101EA
:101D2000E3A906D00201E00E4F6F000E506F05D000
:101D30000201C00E4F6F000E506F0101E3A1E37965
:101D4000E3A706D00201800E4D6F000E4E6F05D046
:101D50000201A00E4D6F000E4E6FC9CF53F24DC25F
:101D6000E9FF4EC2EAFF4D2B000E4E23EF50C96E25
:101D700012009E96C9CF53F202015251000823E28D
:101D80004FC2E9FF50C2EAFF4F2B000E502353C24F
:101D9000EFFF4DC2E9FF4EC2EAFF4D2B4E23EFCFBE
:101DA00053F253C2C9FF520752510CE10101020E16
:101DB000C16F0101E393E381770ED76E470ED66EB4
:101DC000F294D58E01D0C96A1200D9CFE6FFE1CFD7
:101DD000D9FF0101E3A117D0FD0EDBCFE6FFFE0E18
:101DE000DBCFE6FF31EC1BF0E552E5529D96010199
:101DF000E3919D860F0E0001165D05E0B9C1E6FF77
:101E00007BEC1AF0E552E552E7CFD9FF1200D9CFAB
:101E1000E6FFE1CFD9FF0101E3B332D0FD0EDBCF06
:101E2000E9FFFE0EDBCFEAFF1E0EE926000EEA22D6
:101E3000EF50020809E1FD0EDBCFE6FFFE0EDBCF1F
:101E4000E6FF69D8E552E552FD0EDBCFE9FFFE0E55
:101E5000DBCFEAFF150EE926000EEA22EF9EFD0E0B
:101E6000DBCFE6FFFE0EDBCFE6FF9FEC1AF0E5527C
:101E7000E5529D960101E377E3839D860101C02B26
:101E8000E552E7CFD9FF12009D960101E3919D86AF
:101E90001200D9CFE6FFE1CFD9FF0001166BD95070
:101EA000FD0FE96EFF0EDA20EA6E010EEE1801E179
:101EB000ED5002E1168101D0BA6AD950FB0FE96EEC
:101EC000FF0EDA20EA6E010EEE1801E1ED5002E19C
:101ED000168301D0B76AD950F90FE96EFF0EDA20E8
:101EE000EA6E010EEE1801E1ED5002E1168501D017
:101EF000736AD950F70FE96EFF0EDA20EA6E010E11
:101F0000EE1801E1ED5002E1168701D0706AE5524A
:101F1000E7CFD9FF1200D9CFE6FFE1CFD9FFFD0E01
:101F2000DBCFE9FFFE0EDBCFEAFF1C0EE926000E39
:101F3000EA22EF6AFD0EDBCFE9FFFE0EDBCFEAFF00
:101F4000170EE926000EEA22EF6AC6AE0ED0C69E34
:101F5000FD0EDBCFE9FFFE0EDBCFEAFF170EE92611
:101F6000000EEA22010EEF6E22D0F150800B10E03D
:101F7000F250080B0DE0FD0EDBCFE9FFFE0EDBCFCC
:101F8000EAFF170EE926000EEA22020EEF6E0FD0CE
:101F9000F0A60DD0909EFD0EDBCFE9FFFE0EDBCF4D
:101FA000EAFF170EE926000EEA22030EEF6E250E59
:101FB000C614250819E0FD0EDBCFE9FFFE0EDBCFCE
:101FC000EAFF1C0EE926000EEA22010EEF6EFD0E5E
:101FD000DBCFE9FFFE0EDBCFEAFF170EE926000E8E
:101FE000EA22C6CFEFFF80D1C55019E0FD0EDBCF4E
:101FF000E9FFFE0EDBCFEAFF1C0EE926000EEA2207
:10200000020EEF6EFD0EDBCFE9FFFE0EDBCFEAFF27
:10201000170EE926000EEA22C5CFEFFF65D1D0BE2C
:1020200019D0FD0EDBCFE9FFFE0EDBCFEAFF1C0E61
:10203000E926000EEA22030EEF6EFD0EDBCFE9FF6C
:10204000FE0EDBCFEAFF170EE926000EEA22D0CF04
:10205000EFFF4AD19DB619D0FD0EDBCFE9FFFE0E92
:10206000DBCFEAFF1C0EE926000EEA22040EEF6E1B
:10207000FD0EDBCFE9FFFE0EDBCFEAFF170EE926F0
:10208000000EEA229DCFEFFF2FD19C5019E0FD0EEC
:10209000DBCFE9FFFE0EDBCFEAFF1C0EE926000EC8
:1020A000EA22050EEF6EFD0EDBCFE9FFFE0EDBCF61
:1020B000EAFF170EE926000EEA229CCFEFFF14D1AB
:1020C000080E9F5C19E0FD0EDBCFE9FFFE0EDBCFB3
:1020D000EAFF1C0EE926000EEA22060EEF6EFD0E48
:1020E000DBCFE9FFFE0EDBCFEAFF170EE926000E7D
:1020F000EA229FCFEFFFF8D0A25019E0FD0EDBCF10
:10210000E9FFFE0EDBCFEAFF1C0EE926000EEA22F5
:10211000070EEF6EFD0EDBCFE9FFFE0EDBCFEAFF11
:10212000170EE926000EEA22A2CFEFFFDDD0A55060
:1021300019E0FD0EDBCFE9FFFE0EDBCFEAFF1C0E40
:10214000E926000EEA22080EEF6EFD0EDBCFE9FF56
:10215000FE0EDBCFEAFF170EE926000EEA22A5CF1E
:10216000EFFFC2D0100EF214100819E0FD0EDBCF05
:10217000E9FFFE0EDBCFEAFF1C0EE926000EEA2285
:10218000090EEF6EFD0EDBCFE9FFFE0EDBCFEAFF9F
:10219000170EE926000EEA22F2CFEFFFA5D0470E78
:1021A000F11419E0FD0EDBCFE9FFFE0EDBCFEAFFF5
:1021B0001C0EE926000EEA220A0EEF6EFD0EDBCFA2
:1021C000E9FFFE0EDBCFEAFF170EE926000EEA223A
:1021D000F1CFEFFF89D0C00EF01419E0FD0EDBCF78
:1021E000E9FFFE0EDBCFEAFF1C0EE926000EEA2215
:1021F0000B0EEF6EFD0EDBCFE9FFFE0EDBCFEAFF2D
:10220000170EE926000EEA22F0CFEFFF6DD092A85C
:1022100019D0FD0EDBCFE9FFFE0EDBCFEAFF1C0E6F
:10222000E926000EEA220C0EEF6EFD0EDBCFE9FF71
:10223000FE0EDBCFEAFF170EE926000EEA2292CF50
:10224000EFFF52D093B019D0FD0EDBCFE9FFFE0EA9
:10225000DBCFEAFF1C0EE926000EEA220D0EEF6E20
:10226000FD0EDBCFE9FFFE0EDBCFEAFF170EE926FE
:10227000000EEA2293CFEFFF37D03E0E94141C08D5
:1022800019E0FD0EDBCFE9FFFE0EDBCFEAFF1C0EEF
:10229000E926000EEA220E0EEF6EFD0EDBCFE9FFFF
:1022A000FE0EDBCFEAFF170EE926000EEA2294CFDE
:1022B000EFFF1AD097BE18D0FD0EDBCFE9FFFE0E60
:1022C000DBCFEAFF1C0EE926000EEA220F0EEF6EAE
:1022D000FD0EDBCFE9FFFE0EDBCFEAFF170EE9268E
:1022E000000EEA2297CFEFFFE552E7CFD9FF1200A9
:1022F00031DAFD0EDB0403E0FD0EDB504CE1FE0E97
:10230000DB50100A44E01F0A40E0010A3CE0030AE7
:1023100038E0010A31E0070A2DE0010A29E0030A4A
:1023200024E0010A20E00F0A1CE0010A18E0030A79
:1023300011E0010A0CE0070A08E0010A04E0030AC0
:102340002AE128DA08D023DA06D00DDA04D0F9D948
:10235000F70E01D02ADA9214F310926E1CD01ADA1A
:102360000CD015DA0AD0FFD908D0EBD9F70E05D07A
:102370002EDA03D01ADA01D02EDA9714F310976E02
:102380000AD025DA05D011DA03D025DA01D026DA11
:102390009914F310996EE3D1DDD923EC26F0FE0EEB
:1023A000DB50100A3CE01E0A38E0030A34E0010A60
:1023B00030E0070A2CE0010A28E0030A24E0010AC1
:1023C00020E00F0A1CE0010A18E0030A14E0010AE9
:1023D00010E0070A0CE0010A08E0030A04E0010A21
:1023E00022E1E6681ED0FE0E1BD0FD0E19D0FC0EB9
:1023F00017D0FB0E15D0FA0E13D0F90E11D0F80E2F
:102400000FD0F70E0DD0F60E0BD0F50E09D0F40E4E
:1024100007D0F30E05D0F20E03D0F10E01D0F00E6E
:10242000E66E1FD9E552FD0EDBCFE6FF010E8DD91A
:10243000FC0EDBCFE6FF020E88D9FB0EDBCFE6FFFA
:10244000030E83D9FA0EDBCFE6FF040E7ED9F90E18
:10245000DBCFE6FF050E79D9F80EDBCFE6FF060EDF
:1024600074D9F70EDBCFE6FF070E6FD9F60EDBCF80
:10247000E6FF080E6AD9F50EDBCFE6FF090E65D937
:10248000F40EDBCFE6FF0A0E60D9F30EDBCFE6FFDA
:102490000B0E5BD9F20EDBCFE6FF0C0E56D9F10E18
:1024A000DBCFE6FF0D0E51D9F00EDBCFE6FF0E0EAF
:1024B0004CD9EF0EDBCFE6FF0F0E47D9EE0EDBCF88
:1024C000E6FF100E42D94BD145D9FE0EDB50100A63
:1024D00044E01F0A40E0010A3CE0030A38E0010A38
:1024E00031E0070A2DE0010A29E0030A24E0010A8D
:1024F00020E00F0A1CE0010A18E0030A11E0010ABB
:102500000CE0070A08E0010A04E0030A2BE142D9C3
:1025100008D03DD906D027D904D013D9F70E01D061
:1025200044D98914F310896E1FD034D90CD02FD917
:102530000AD019D908D005D9F70E05D048D903D04B
:1025400034D901D048D98E14F3108E6E0DD03FD9F6
:1025500005D02BD903D03FD901D040D99014F31026
:10256000906E02D0FE0EDB50FAD0F4D8FE0EDB5097
:10257000100A57E01F0A51E0010A4BE0030A45E048
:10258000010A3FE0070A39E0010A33E0030A2DE0BF
:10259000010A27E00F0A21E0010A1CE0030A16E005
:1025A000010A10E0070A0AE0010A04E0030A3EE11A
:1025B000805011D08050020B3AE036D08050040B8E
:1025C00036E032D08050080B32E02ED08050200B05
:1025D0002EE02AD08550010B2AD08550020B27E02F
:1025E00023D08550040B23E01FD08550080B1FE03B
:1025F0001BD08550100B1BE017D08550200B17E027
:1026000013D08550400B13E00FD08750100B0FE014
:102610000BD08750200B0BE007D08750400B07E012
:1026200003D08750800B03E0010E01D0000E97D03D
:1026300091D8E66AFE0EDBCFE6FF5ADEE552E552A0
:10264000FD0EDBCFE6FFFE0EDBCFE6FF3DDFE55202
:10265000E55285D07FD8E66AADD07CD8010EE66E13
:10266000A9D078D8FE0EDBCF6BF279D073D8020EEA
:10267000E126F29CFE0EDB507F0B79D807EC04F0CC
:102680000009FCE14AEC29F0D7EC29F0C4502D6E8A
:102690002E6E2D6AC35000012D102B6E2EC02CF013
:1026A000DE6E2EC0DDFFF28CDECF2BF0DDCF2CF006
:1026B0002BC0F3FF2CC0F4FFD9CFE1FF50D04AD894
:1026C000030EE126010EF36EFE0EDBCFF4FFF35096
:1026D000F45C04E3FE0EDB50100803E2F36AF46AD4
:1026E0002DD0FE0EDB50F76A850FF66E530EF722E3
:1026F0000800F550DF6EF29C7F0EDF1438D807EC2F
:1027000004F00009FCE14AEC29F0D7EC29F0C450B0
:102710002E6E2D6AC3502D102B6E010E2BC0DBFFC9
:10272000020E2EC0DBFFF28C010EDBCF2BF0020E6F
:10273000DBCF2CF02BC0F3FF2CC0F4FFD9CFE1FF8F
:102740000ED03FD8F346F3461200E66ED1DDE552D7
:10275000E5521200D9CFE6FFE1CFD9FF1200E552D2
:10276000E7CFD9FF12002DD8F346FB0E1200FE0B67
:10277000FD0BE66E6BC2E6FF58EC28F0E552E55221
:102780000A0EE66EAFEC29F0E552DAEF29F019D81F
:10279000FD0E1200FD0EDB50010BF36EFE0E12005B
:1027A000F346F346F346BF0E1200CBDFF346F34683
:1027B000DF0E1200FE0EDBCFE6FF3ADFE552E552F8
:1027C000CED7FD0EDB50010BF36EF3461200B9DFDE
:1027D000F346EF0E1200B5DFD0EF13F0B2DFF34691
:0A27E000F346F346F3467F0E1200A5
:0627EA001FDA1A0EE126C1
:1027F000D9CF2BF0DACF2CF03CDA0101AA0E886F8A
:10280000550E896F1E0E8A6F120E8B6F8C6BFE0E2B
:10281000DB5005E0FE0EDB0402E0000E65D0FE0E8C
:10282000DB5001E08C810701F25101018C13050E90
:10283000F36E190EF3CFDBFF150EE8D906E2EDD9E2
:10284000200EEF6E190EDB2AF7D7190EDB6A100E79
:10285000DDD913E2CDD90F01F8D9EF50E66E190E8C
:10286000DB50050FEA6A880FE96E010EEA22E55295
:10287000E750EF6E190EDB2AEAD701019E6B040EBA
:10288000F36E190EF3CFDBFF150EC0D906E2C5D9E2
:10289000EF509E27190EDB2AF7D79E1D010F9E6F62
:1028A000E8CF9DF1190EDB6A160EB0D909E2B5D951
:1028B000EF50E66E92EC23F0E552190EDB2AF4D7C6
:1028C000F1C72BF02C6A2D6A2E6AF1C7E6FF2CC0E7
:1028D000E6FF2DC0E6FF2EC0E6FFFAEC0CF0E55255
:1028E000E552E552E552010ED9CFE1FFA3D1080E22
:1028F0000701EE5D03E1F29CEE6BF28C120095D9BC
:10290000E6520701EE51080A57E00C0A2EE0070ACA
:1029100023E0010A11E0030A08E0010A4CE1FE0E7F
:10292000DB50AA0849E1010E3FD0EE6BFE0EDB50F2
:10293000550842E1020E38D00101A06BA0C1F0F7AA
:10294000A0C19FF1FE0EDBCFEFF70701EE6B160E75
:10295000EF5D32E1030E28D0FE0EDBCFF0F7EE6B19
:10296000020EF05D29E1040E1FD001019F519F2B43
:10297000EA6A5A0FE96E010EEA22FE0EDBCFEFFF84
:102980000701F007F05112E1FE0EDB500101A02714
:10299000A05112E15AC166F166B1678166B36783DF
:1029A00066B567850701080EEE6F06D0FE0EDB5098
:1029B0000101A02701D0EE6BE5523CD152D90701AD
:1029C000EE6B0101666B676BFE0EE66E280EE66E1F
:1029D000BFEC23F0E552E552120031EF16F025D995
:1029E000E66A03DFE552F29CD950FD0F27D90DE0CE
:1029F000010E0101671502E0010E01D0000EE66E26
:102A0000FD0EDBCFE9FFFE0E26D9D950FB0F16D9FC
:102A10000DE0020E0101671502E0010E01D0000E6B
:102A2000E66EFB0EDBCFE9FFFC0E15D9D950F90F8E
:102A300005D90DE0040E0101671502E0010E01D079
:102A4000000EE66EF90EDBCFE9FFFA0E04D907019E
:102A5000EE6B0101676BF28CEDD0E7D8020EE12638
:102A6000800EE66EFC0EE66EF4EC27F0E552E552C1
:102A7000A59AA598989298846E50DF6E6E50DF6E7E
:102A8000A49A0701F26B010EDB6A100EF36E010EC1
:102A9000DBCFF4FFF350F45C15E2010EDB50EA6A81
:102AA000680FE96E010EEA22200EEF6E010EDB5078
:102AB000EA6A780FE96E010EEA22200EEF6E010E2F
:102AC000DB2AE3D7D9CFE1FFB5D0AFD81D0EE12681
:102AD000D0D8D950FC0F2B6EFF0EDA202C6E1B0EB7
:102AE0002BC0DBFF1C0E2CC0DBFF1B0EDBCFE6FF79
:102AF0001C0EDBCFE6FFFC0EDBCF2BF0FD0EDBCF99
:102B00002CF02D6A2BC0E6FF2CC0E6FF2DC0E6FF9F
:102B1000D950170FE66E000EDA20E66E50EC04F086
:102B2000F56E070EE15EF5501A0EF3CFDBFF170EC0
:102B3000DBCFE9FF180EDBCFEAFFEF6A1A0EDB509E
:102B4000100805E2100EF36E1A0EF3CFDBFFFE0E37
:102B5000DB5005E0FE0EDB0402E0000E2FD0190E64
:102B6000DB6A100E53D808E243D80F016ED8200E4E
:102B7000EF6E190EDB2AF5D7190EDB6A1A0EDB5041
:102B800045D816E2D9CF2DF0DACF2EF0190EDB5052
:102B90000F01D924E96E000EDA20EA6EEF50E66EDE
:102BA00027D853D8E552E750EF6E190EDB2AE6D747
:102BB000FE0EDBCFE6FF19DEE552010ED9CFE1FFB5
:102BC00039D033D8FE0EDB5005E0FE0EDB0402E008
:102BD000000E0DD0FE0EDB5004E00701020EF26F76
:102BE00002D00701F26BE66A00DEE552010E22D048
:102BF000FE0EDB50100DF3CF2BF0F4CF2CF0680E4F
:102C00002B26010E2C22190EDB501200F36E190E2A
:102C1000DBCFF4FFF350F45C1200190EDB50EA6ACC
:102C2000880FE96E010EEA221200D9CFE6FFE1CF4C
:102C3000D9FF1200E552E7CFD9FF1200E96EFF0E6F
:102C4000DA20EA6EEE50ED1012002B24E96E000E31
:102C50002C20EA6E1200DBCFEAFFE552E750EF6E60
:102C60001200000EE66EE66ABFEC23F0E552E55274
:102C70001200170ED9CFDBFF180EDACFDBFF1200E0
:102C8000D9CFE6FFE1CFD9FF020EE12616EE00F024
:102C900026EE00F0F86A269CA68EA69C53EC1AF04D
:102CA000D4EC25F0C5EC1CF00701B66BB76BB86B24
:102CB000B96B02016E5101E1FCD70101E251E66EF0
:102CC000E66ADF0E2B6E420E2C6E2D6A2BC0E6FFDD
:102CD0002CC0E6FF2DC0E6FFBBEC26F0F56E050E1E
:102CE000E15EF55002013E5114E102013F5111E154
:102CF0000101040EB76F640EE66EE66AE66AE66AE4
:102D0000FAEC0CF0E552E552E552E552B8EC28F049
:102D1000ADD1FF0E02013E5D01E0B8D0080E010109
:102D2000E25D22E20101E251E66EE66AA60E2B6E3A
:102D3000420E2C6E2D6A2BC0E6FF2CC0E6FF2DC084
:102D4000E6FFBBEC26F0F56E050EE15EF550E80EF1
:102D5000E66E030EE66EE66AE66AFAEC0CF0E55201
:102D6000E552E552E552DED70101D5510CE1640E82
:102D7000E66EE66AE66AE66AFAEC0CF0E552E552BF
:102D8000E552E552F1D78A0E2B6E420E2C6E2D6A5B
:102D90002BC0E6FF2CC0E6FF2DC0E6FFBBEC26F003
:102DA000E552E552E552640EE66EE66AE66AE66AC8
:102DB000FAEC0CF0E552E552E552E55203EC04F072
:102DC00078EC1CF0000901E1FBD7C3EC0AF01BC052
:102DD000B6F71CC0B7F71DC0B8F71EC0B9F75CEC5A
:102DE0001CF000092DE0640EE66EE66AE66AE66A0B
:102DF000FAEC0CF0E552E552E552E5520101020E03
:102E0000B76F51EC1CF05CEC1CF0000901E0FBD743
:102E100001017F0EA76F01017F0EA86F01017F0ED8
:102E2000A96F01017F0EAA6F01017F0EAB6F010137
:102E30007F0EAC6F01017F0EAD6F01017F0EAE6F93
:102E40000101B76BE66AE66AE66AE66ACBEC29F04E
:102E5000E552E552E552E55201017F0EA76F0101EF
:102E60007F0EA86F01017F0EA96F01017F0EAA6F6F
:102E700001017F0EAB6F01017F0EAC6F01017F0E70
:102E8000AD6F01017F0EAE6FAAD7F0D0640EE66E73
:102E9000E66AE66AE66AFAEC0CF0E552E552E552BB
:102EA000E55203EC04F00101C55101E1FCD7C3EC8C
:102EB0000AF01BC0B6F71CC0B7F71DC0B8F71EC09C
:102EC000B9F70101D55121E00101E25107081DE2E6
:102ED000360E2B6E420E2C6E2D6A2BC0E6FF2CC0D8
:102EE000E6FF2DC0E6FFBBEC26F0E552E552E552C9
:102EF000E80EE66E030EE66EE66AE66AFAEC0CF0A1
:102F0000E552E552E552E552E3D702013F51E66E44
:102F1000E66A02013E51E66EE66AE70E2B6E410E4E
:102F20002C6E2D6A2BC0E6FF2CC0E6FF2DC0E6FFFD
:102F3000BBEC26F0F56E070EE15EF55002013E5146
:102F400042E05CEC1CF000093EE0640EE66EE66ACE
:102F5000E66AE66AFAEC0CF0E552E552E552E55213
:102F60000101020EB76F3EC22BF02C6A2D6A2E6A49
:102F70002BC0E6FF2CC0E6FF2DC0E6FF2EC0E6FF0B
:102F8000D1EC29F0E552E552E552E5525CEC1CF03B
:102F9000000901E0FBD701017F0EA76F01017F0E41
:102FA000A86F01017F0EA96F01017F0EAA6F0101B9
:102FB0007F0EAB6F01017F0EAC6F01017F0EAD6F15
:102FC00001017F0EAE6F02013F5150E00701B66B69
:102FD000B76BB86BB96B020140693FC23EF2C3ECFC
:102FE0000AF01BC0B6F71CC0B7F71DC0B8F71EC06B
:102FF000B9F7640EE66EE66AE66AE66AFAEC0CF089
:10300000E552E552E552E5520101B76B3FC22BF0A4
:103010002C6A2D6A2E6A2BC0E6FF2CC0E6FF2DC05D
:10302000E6FF2EC0E6FFCBEC29F0E552E552E55273
:10303000E5525CEC1CF0000901E0FBD701017F0EBA
:10304000A76F01017F0EA86F01017F0EA96F01011B
:103050007F0EAA6F01017F0EAB6F01017F0EAC6F77
:1030600001017F0EAD6F01017F0EAE6FE80EE66EBF
:10307000030EE66EE66AE66AFAEC0CF0E552E552FB
:10308000E552E552F3D70AD6D9CFE1FFE552E7CFB3
:04309000D9FF120052
:0C309400D8CFE4FFE0CFE4FFE46EDACF19
:1030A000E4FFE2CFDAFFE9CFE4FFEACFE4FFF3CFBA
:1030B000E4FFF4CFE4FF00EE17F0140EE80403E39E
:1030C000EECFE4FFFBD700EE2BF00B0EE80403E39A
:1030D000EECFE4FFFBD7E652E1D9030EE126A45080
:1030E000200B05E0A350200B02E0CDEC23F09EA0C6
:1030F00003D09E90C5EC0BF09E50200B05E09D5038
:10310000200B02E0A7EC23F09E50100B05E09D5031
:10311000100B02E0FBEC23F0A450100B05E0A350D1
:10312000100B02E00DEC24F0F050020B15E0F05013
:10313000100B12E00201585159110DE0F8C1E6FFE1
:10314000010EE66E05D059C2FAFF02015851F96E20
:10315000FADFE552E552F092F050040B15E0F05022
:10316000200B12E002015A515B110DE0F9C1E6FF9C
:10317000020EE66E05D05BC2FAFF02015A51F96EEB
:10318000FADFE552E552F094F250010B01E18AD0EA
:10319000F250080B01E186D08150DF6EF290DF50D3
:1031A00002016419E76E010EE7CFDBFFDFCF64F2A7
:1031B000DBA81BD05C515D1118E0100EDF1402E09B
:1031C000010E01D0000E49D90101FA5D0EE1020E97
:1031D000DBCFE6FF030EE66E05D05DC2FAFF02010B
:1031E0005C51F96EFADFE552E552010EDBAA1CD004
:1031F00002015E515F1118E0200EDF1402E0010EA3
:1032000001D0000E2AD90101FB5D0EE1020EDBCFD9
:10321000E6FF040EE66E05D05FC2FAFF02015E51C2
:10322000F96EFADFE552E552010EDBAC1CD002016B
:103230006051611118E0400EDF1402E0010E01D070
:10324000000E0BD90101FC5D0EE1020EDBCFE6FFA3
:10325000050EE66E05D061C2FAFF02016051F96EFB
:10326000FADFE552E552010EDBAE1CD002016251DD
:10327000631118E0800EDF1402E0010E01D0000E91
:10328000ECD80101FD5D0EE1020EDBCFE6FF060E7C
:10329000E66E05D063C2FAFF02016251F96EFADFF1
:1032A000E552E552D9CFE1FFE552E7CFD9FFE5522C
:1032B00000EE35F00B0EE80403E3E5CFEDFFFBD79E
:1032C00000EE2AF0140EE80403E3E5CFEDFFFBD790
:1032D000E5CFF4FFE5CFF3FFE5CFEAFFE5CFE9FF68
:1032E000E5CFDAFFE550E5CFE0FFE5CFD8FF1000EE
:1032F000F09EF192F19081CF64F2F290F28612008A
:10330000B2D841E0030A34E0010A27E0070A1AE0D4
:10331000010A0DE0030A42E1FB0EDBCF58F2FC0E7E
:10332000DBCF59F2938491D8A4D8F08839D0FB0E22
:10333000DBCF5AF2FC0EDBCF5BF2938686D8A2D8A5
:10334000F08A2ED0FD0EDBCFFAF1FB0EDBCF5CF264
:10335000FC0EDBCF5DF2938823D0FD0EDBCFFBF1BB
:10336000FB0EDBCF5EF2FC0EDBCF5FF2938A18D050
:10337000FD0EDBCFFCF1FB0EDBCF60F2FC0EDBCFF2
:1033800061F2938C0DD0FD0EDBCFFDF1FB0EDBCF98
:1033900062F2FC0EDBCF63F2938E02D0FE0EDB50A6
:1033A000F28C78D07BD8FE0EDB50060A1CE0030AB4
:1033B00016E0010A10E0070A0AE0010A05E0030A24
:1033C00015E143D856D812D040D85CD80FD0FD0EA6
:1033D000DBCFFAF10BD0FD0EDBCFFBF107D0FD0EFA
:1033E000DBCFFCF103D0FD0EDBCFFDF153D03BD89A
:1033F00020E0030A1AE0010A14E0070A0EE0010ABD
:1034000007E0030A1AE1F0980201586B596B17D0D4
:10341000F09A02015A6B5B6B12D002015C6B5D6B20
:103420000ED002015E6B5F6B0AD00201606B616BB4
:1034300006D00201626B636B02D0FE0EDB50F28C91
:1034400029D01200120012001200FD0EDB50010BF9
:10345000F36EF346F346F3461200E76E020EE7CF33
:10346000DBFFDB5012001AD8F29CFE0EDB50060A7E
:103470001200F346EF0EF114F310F16EFD0EDBCFE8
:10348000F8F11200F70EF114F310F16EFD0EDBCF20
:10349000F9F11200E552E7CFD9FF1200D9CFE6FFCC
:0634A000E1CFD9FF12008C
:0A34A600000EE96EEA6E040060EC0F
:1034B0001AF0EA2A080EEA5CD8A456EF1AF01200B5
:1034C000EF6AE93E60EF1AF01200FF0EE3CF09F059
:1034D00009380F0B060FD8B2070F2A0FAD6E38EC64
:1034E00024F009500F0B060FD8B2070F2A0FAD6E4C
:1034F00038EC24F0000CFF0EE3CF15F015B0968EDB
:1035000015A0969E15B2988015A2989015B498862D
:1035100015A4989615B6988815A6989815B896800B
:1035200015A8969015BA968215AA969215BC9684FF
:1035300015AC969415BE968615AE96961200EACFF7
:1035400004F0E9CF05F0FF0EE3CFEAFFFE0EE3CF74
:10355000E9FFE3A741D0EECFA0F0EECFA1F0EECF90
:10356000A2F0EECFA3F0EECFA4F0EECFA5F0EECF19
:10357000A6F0EECFA7F0EECFA8F0EECFA9F0EECFF9
:10358000AAF0EECFABF0EECFACF0EECFADF0EECFD9
:10359000AEF0EECFAFF0EECFB0F0EECFB1F0EECFB9
:1035A000B2F0EECFB3F0EECFB4F0EECFB5F0EECF99
:1035B000B6F0EECFB7F0EECFB8F0EECFB9F0EECF79
:1035C000BAF0EECFBBF0EECFBCF0EECFBDF0EECF59
:1035D000BEF0EECFBFF040D0EECF80F0EECF81F066
:1035E000EECF82F0EECF83F0EECF84F0EECF85F019
:1035F000EECF86F0EECF87F0EECF88F0EECF89F0F9
:10360000EECF8AF0EECF8BF0EECF8CF0EECF8DF0D8
:10361000EECF8EF0EECF8FF0EECF90F0EECF91F0B8
:10362000EECF92F0EECF93F0EECF94F0EECF95F098
:10363000EECF96F0EECF97F0EECF98F0EECF99F078
:10364000EECF9AF0EECF9BF0EECF9CF0EECF9DF058
:10365000EECF9EF0EECF9FF004C0EAFF05C0E9FF79
:103660001200E3A11200EACF04F0E9CF05F0FF0E4B
:10367000E3CFEAFFFE0EE3CFE9FFE3A941D0C0C0EC
:10368000EEFFC1C0EEFFC2C0EEFFC3C0EEFFC4C07C
:10369000EEFFC5C0EEFFC6C0EEFFC7C0EEFFC8C05C
:1036A000EEFFC9C0EEFFCAC0EEFFCBC0EEFFCCC03C
:1036B000EEFFCDC0EEFFCEC0EEFFCFC0EEFFD0C01C
:1036C000EEFFD1C0EEFFD2C0EEFFD3C0EEFFD4C0FC
:1036D000EEFFD5C0EEFFD6C0EEFFD7C0EEFFD8C0DC
:1036E000EEFFD9C0EEFFDAC0EEFFDBC0EEFFDCC0BC
:1036F000EEFFDDC0EEFFDEC0EEFFDFC0EEFF40D02C
:10370000E0C0EEFFE1C0EEFFE2C0EEFFE3C0EEFF7F
:10371000E4C0EEFFE5C0EEFFE6C0EEFFE7C0EEFF5F
:10372000E8C0EEFFE9C0EEFFEAC0EEFFEBC0EEFF3F
:10373000ECC0EEFFEDC0EEFFEEC0EEFFEFC0EEFF1F
:10374000F0C0EEFFF1C0EEFFF2C0EEFFF3C0EEFFFF
:10375000F4C0EEFFF5C0EEFFF6C0EEFFF7C0EEFFDF
:10376000F8C0EEFFF9C0EEFFFAC0EEFFFBC0EEFFBF
:10377000FCC0EEFFFDC0EEFFFEC0EEFFFFC0EEFF9F
:1037800004C0EAFF05C0E9FF1200F2B412001650AF
:103790000F0AD8B41200FF0EE3CF0AF0FE0EE3CFFB
:1037A0000BF0FD0EE3CF0CF0FC0EE3CF0DF00A2A78
:1037B00016A08D8E0B2A16A28F800C2A16A48F8637
:1037C0000D2A16A68F88FB0EE3CF0EF0FA0EE3CF7C
:1037D0000FF0F90EE3CF10F0F80EE3CF11F00E2A40
:1037E0008D800F2A8D82102A8D84112A8D8628ECD7
:1037F0001CF00A2EFEEF1BF016A08D9E0B2E03EF81
:103800001CF016A28F900C2E08EF1CF016A48F96B9
:1038100000000D2E0EEF1CF016A68F9800000E2E45
:1038200013EF1CF08D9000000F2E18EF1CF08D92FE
:103830000000102E1DEF1CF08D940000112E22EFC1
:103840001CF08D964AEC1CF0133EF9EF1BF01200B1
:10385000D70E136E000000000000000040EC1CF0CA
:10386000132E2AEF1CF0D70E136E0000000000008C
:10387000000040EC1CF0132E35EF1CF0000012008D
:10388000000043EF1CF000000000000000000000FA
:1038900000001200030E146E0000142E4CEF1CF0FA
:0238A000120014
:0E38A200E66AE66AE66AE66AD1EC29F0E552CB
:1038B000E552E552E552FFD702013E5101E1010C0C
:1038C000FF0E3E5D04E1400E0101D515120081ACF2
:1038D000010C81AE000CD2EC0AF002013E512D6EBB
:1038E0002E6AF3502D5CF4502E5801E2000C010CAE
:1038F000800E0101D51501E0000C010C7FD9FE0EF0
:10390000DB50FF0804E0FD0EDB50FF0804E1FE0E73
:10391000DB68FD0EDB68FE0EDBCF3EF2FD0EDBCF7B
:103920003FF271D16BD90101B969E150FD0F5FD947
:1039300001E1B991D950FB0F5AD901E1B993D9509E
:10394000F90F55D901E1B995D950F70F50D901E1D7
:10395000B99759D153D9F70EDBCFE6FFF80EDBCF7D
:10396000E6FFF90EDBCFE6FFFA0EDBCFE6FFFB0E3C
:10397000DBCFE6FFFC0EDBCFE6FFFD0EDBCFE6FF85
:10398000FE0EDBCFE6FF50D93ED138D9E652020118
:103990003E6B0201406943EC0EF09784978297805A
:1039A000928A9286928492829280F70EE66E31EC31
:1039B00013F0E552998E998C998A9988978C978AF9
:1039C00097889786010EE66EE66AE66EE66AE66E10
:1039D000E66AE66EE66A28D9EEEC24F0150EE66E8D
:1039E000010EE66E2CEC23F0E552E55278EC19F06E
:1039F0004BEC0AF00CD985EC0EF02AEC29F0E552DC
:103A000002D10101C3511200C30EE66E010EE66E33
:103A1000E5EC0EF0E552E5520201010E6E6F07EF84
:103A20001EF0ECD8080EE126FE0EDB500EE101017F
:103A3000D651E66EE66AE251E66EE66AE80E2B6E55
:103A4000400ECCD8F56E070EBCD0FE0EDB046BE149
:103A50000101D55104E1DB0E2B6E400EB8D0010EF2
:103A6000D51502E0010E01D0000EDF6E020ED51555
:103A700002E0010E01D0000EE76E010EE7CFDBFF82
:103A8000040ED51502E0010E01D0000EE76E020E05
:103A9000E7CFDBFF080ED51502E0010E01D0000EC6
:103AA000E76E030EE7CFDBFF100ED51502E0010E27
:103AB00001D0000EE76E040EE7CFDBFF200ED51518
:103AC00002E0010E01D0000EE76E050EE7CFDBFF2E
:103AD000400ED51502E0010E01D0000EE76E060E75
:103AE000E7CFDBFF800ED51502E0010E01D0000EFE
:103AF000E76E070EE7CFDBFF93D8060E91D8050ED1
:103B00008FD8040E8DD8030E8BD8020E89D8010EE3
:103B100087D8DFCFE6FFE66ABC0E2B6E400E5ED87C
:103B2000F56E130E4ED0FE0EDB5002084DE1800EF6
:103B30000101D51502E0010E01D0000E2B6E2C6A9A
:103B40002BBE2C682BC0E6FF2CC0E6FF400ED5151F
:103B500002E0010E01D0000E2D6E2E6A2DBE2E68E1
:103B60002DC0E6FF2EC0E6FF080ED51502E0010EBF
:103B700001D0000E2F6E306A2FBE30682FC0E6FFD6
:103B800030C0E6FF040ED51502E0010E01D0000E94
:103B9000316E326A31BE326831C0E6FF32C0E6FFB4
:103BA000D551E66EE66A760E336E400E346E356A97
:103BB00033C0E6FFE66E35C0E6FFBBEC26F0F56EDF
:103BC0000D0EE15EF55007D0680E2B6E400E06D844
:103BD000E552E552E552D9CFE1FF15D02C6E2D6AA2
:103BE0002BC0E6FFE66E2DC0E6FFBBEF26F0E96EC8
:103BF000FF0EDA20EA6EEE50ED101200D9CFE6FF8C
:103C0000E1CFD9FF1200E552E7CFD9FF1200A30E92
:103C1000E66E010EE66E07EC0FF0E552E55212007B
:103C2000DBCFE6FFE66A12007DDEF56E080EE15E90
:043C3000F550120039
:0C3C340071D9FD0EDBCF2CF00001800EDA
:103C40002C140DE1FC0EDBCF2DF0FD0EDBCF2EF0A2
:103C50002E341BE22D50FF08000E2E5416E265D9BB
:103C6000FE0EDBCFE6FFE66A870E2B6E410E2C6E52
:103C70002D6A2BC0E6FFE66E2DC0E6FFBBEC26F0FA
:103C8000F56E070EE15EF55034D0FE0EDB50080AEB
:103C90002AE00F0A24E0010A1EE0030A18E0010AE4
:103CA00012E0070A0CE0010A06E0030A20E1FC0E1C
:103CB000DBCFA7F11ED0FC0EDBCFA8F11AD0FC0E93
:103CC000DBCFA9F116D0FC0EDBCFAAF112D0FC0E8F
:103CD000DBCFABF10ED0FC0EDBCFACF10AD0FC0E8B
:103CE000DBCFADF106D0FC0EDBCFAEF102D0FE0E85
:103CF000DB5017D13FD13ED10FD9FD0EDBCF2BF0DA
:103D0000FE0EDBCF2CF02C3407E22B50FF08000E08
:103D10002C5402E2FF0E0AD0FE0EDBCF2CF0800EF8
:103D20002C1402E0000E02D0FD0EDB50FAD011D9A7
:103D3000F90EDB5003E031D92B50DF6EF80EDB506B
:103D400004E02ED9010E2BC0DBFFDFCFE6FFE66AD1
:103D5000FB0EC6D8010EDBCFE6FFE66AFA0EC0D82E
:103D6000D9CFE1FFDED0F5D8F70EDB5002E1EDD878
:103D700001D013D9CCD8FB0EB3D8F60EDB5002E13C
:103D8000DBD801D00DD9C3D8FA0EAAD8F50EDB5076
:103D900002E1DBD801D001D9BAD8F90EA1D8F40ECE
:103DA000DB5002E1C9D801D0FBD8B1D8F80E98D8C1
:103DB000D9CFE1FFB6D0B0D8FD0E99D80101E66F9A
:103DC000E76B7F0EE65F000EE75BFC0E90D801010B
:103DD000E86FE96B7F0EE85F000EE95BE651E825CE
:103DE000EC6FE751E921ED6FE651E85DEA6FE751CD
:103DF000E959EB6FF90EDB5004E0EA6DEB1F000EA2
:103E0000EB23F80EDB5004E0EC6DED1F000EED230C
:103E10007F0E2C6AEA252B6EEB51A8D8E66EE66A77
:103E2000FB0E5ED87F0E01012C6AEC252B6EED5146
:103E30009DD8E66EE66AFA0E53D873D06DD8FD0EA3
:103E400056D80101EE6FEF6B7F0EEE5F000EEF5B59
:103E5000FC0E4DD80101F06FF16B7F0EF05F000E8C
:103E6000F15BEE51F0252B6EEF51F1219CD8010151
:103E7000F46FF56BEE51F05D2B6EF151EF5593D869
:103E80000101F26FF36BF70EDB5002E078D804D03B
:103E9000F2C1E6FFF3C1E6FFFB0E22D8F50EDB50C0
:103EA00002E06DD804D0F2C1E6FFF3C1E6FFF90EDF
:103EB00017D8F60EDB5002E069D804D0F4C1E6FF53
:103EC000F5C1E6FFFA0E0CD8F40EDB5002E05ED826
:103ED00004D0F4C1E6FFF5C1E6FFF80E01D821D009
:103EE000DBCFE6FFA7DEE552E552E5521200DBCF5D
:103EF000E6FFFE0EDBCFE6FF24EC22F0E552E552B2
:103F00001200FF0ED8802B56000E2C5612002BC02C
:103F1000E6FF2CC0E6FF1200D9CFE6FFE1CFD9FFC4
:103F20001200E552E7CFD9FF1200FC0EDBCFE6FF0F
:103F3000FD0EDBCFE6FF1200010EDB502B6E2C6A6C
:103F40001200DADEE552E5521200DF502B6E2C6AC9
:103F50001200E2DF020EE126FD0EC9DFDF6EFC0E6D
:103F6000C6DFE76E010EE7CFDBFF12002C22CFDFAA
:103F7000A1EF1FF0D1DFD9DFFE0EB2DFD2D7F2C141
:103F80002BF0F3C12CF0BDDF87EF1FF0F4C12BF055
:103F9000F5C12CF0B6DF87EF1FF0D7DF81EF1FF000
:103FA000CBDF81EF1FF02C6E7F0E2B26000EB6EFBD
:023FB0001FF000
:0E3FB20072696768743D25640A006D69646475
:103FC0006C653D25640A006C6566743D25640A00D5
:103FD0004572726F723A20696E76616C6964206115
:103FE0006E616C6F6720706F7274206E756D6265A4
:103FF000722025640D00496C6C6567616C20494F27
:1040000020706F72742025642072657175657374F9
:10401000656400496C6C6567616C20494F20706F66
:104020007274202564207265717565737465640D02
:1040300000496C6C6567616C20706F7274206469F4
:1040400072656374696F6E0054696D6572206E7578
:104050006D6265722028256429206F7574206F6653
:104060002072616E67650D00496E76616C6964202F
:10407000747970650A00776966693A2025642C2096
:10408000776966696163746976653A2025642C20D6
:104090006669656C6463746C3A2025642C206175D4
:1040A000746F6E6F6D6F75733A2025642C20646990
:1040B0007361626C65643A2025640A006F695F6110
:1040C0006E616C6F6731333A202564256425642561
:1040D0006425642564256425640A004C6567616372
:1040E00079206D6F64650A006D61737465725F7627
:1040F000657273696F6E3A202564206F695F616E27
:10410000616C6F6731343A2025640A00556E726520
:1041100067697374657220696E7465727275707404
:104120003A20706F7274202564206973206F757453
:10413000206F662072616E67650D00526567697356
:1041400074657220696E746572727570743A20704D
:104150006F7274202564206973206F7574206F66F8
:104160002072616E67650D0053657474696E672017
:1041700050574D2077697468206261642076616CC5
:1041800075652025640A0043616E6E6F7420736547
:104190007420746865204D6F746F72202564205000
:1041A000574D20746F2025642E2056616C75652054
:1041B00052616E676520697320302E2E3235350DC1
:1041C00000496E76616C6964204F4920506F7274AB
:1041D0000D00496E76616C6964204F492046756E0A
:1041E0006374696F6E0D004372797374616C204360
:1041F0006F6D7065746974696F6E2050726F6A6557
:1042000063742E204175746F6E6F6D6F75732054DB
:10421000696D653A202564207365632E204F7065B3
:104220007261746F722054696D653A202564207341
:1042300065632E0D0D0043616E6E6F742062652004
:1042400072756E20776974682057694669206465C5
:10425000766963652E20506C6561736520636F6EAF
:104260006E656374204372797374616C20616E644F
:1042700020726573746172742074686520636F6E58
:1042800074726F6C6C65722E0A0057694669204320
:104290006F6D7065746974696F6E2050726F6A65B6
:1042A00063742E0D0D004D617374657220636F642D
:1042B000652076657273696F6E3A2025642E2050F2
:1042C0006C656173652075706461746520746865E0
:1042D000206D617374657220636F64652E0A004DF2
:1042E000617374657220636F6465207665727369AB
:0942F0006F6E3A2025640D0D00EB
:0642FA0066D9020EE12668
:10430000FE0EDB0402E1010E07D0FE0EDB500208B8
:1043100002E1020E01D0030EDF6EDF500101C51570
:10432000E76E010EE7CFDBFFDB5002E1000E01D0AC
:10433000010ED9CFE1FF4DD147D9FE0EDB5022E16E
:104340000101C551010B03E1C551020B06E0C55146
:10435000010B05E0C551020B02E1010E0FD0C55162
:10436000010B05E1C551020B02E0020E07D0C55159
:10437000010B08E0C551020B05E0010EF36EFE0EC5
:10438000F3CFDBFFFE0EDB5024D11ED9E652DF6AED
:1043900010D9020A28E0030A54E1FD0EDB50040A9A
:1043A0001DE0070A12E0010A0BE0030A4AE10101DD
:1043B000CD512B6E2C6A2C342DE201D935E32AD055
:1043C000370E0101CD5D26E22FD00101CE512B6EBB
:1043D0002C6A2C341FE2F3D827E31CD0370E0101DE
:1043E000CE5D18E221D0FD0EDB50040A22E0070A60
:1043F00013E0010A0BE0030A24E10101D3512B6E03
:104400002C6A2C3407E2DBD80FE304D0370E01010D
:10441000D35D0AE3000E0BD00101D4512B6E2C6A40
:104420002C3404E2CCD802E2010E01D0000EDF6E83
:1044300008D0370E0101D45D02E2010E01D0000E5A
:10444000DF6EDF50E552C5D0BFD8E6527F0EDF6E7B
:10445000020E0101B75D0AE0040EB75D09E001013B
:10446000C551010B05E1C551020B02E1DF5045D0FA
:10447000A0D8020A22E0030A3FE1FD0EDB50060A43
:1044800019E0030A14E0010A0FE0070A0AE0010A32
:1044900005E0030A31E1C9C1DFFF2ED0CAC1DFFF49
:1044A0002BD0CBC1DFFF28D0CCC1DFFF25D0CDC1C1
:1044B000DFFF22D0CEC1DFFF1FD0FD0EDB50060A8A
:1044C00019E0030A14E0010A0FE0070A0AE0010AF2
:1044D00005E0030A11E1CFC1DFFF0ED0D0C1DFFF3D
:1044E0000BD0D1C1DFFF08D0D2C1DFFF05D0D3C1CF
:1044F000DFFF02D0D4C1DFFFDF50E5526AD064D8BD
:10450000FD0EDBCFE6FF55D8E66E9EDFE552E552A5
:1045100060D02ED801E042D834D02AD801E03ED86D
:1045200030D026D801E03AD82CD04ED8FD0EDBCFC3
:10453000E9FFFE0EDBCFEAFFBFC1EFFFFB0EDBCFD3
:10454000E9FFFC0EDBCFEAFFBAC1EFFF42D03CD857
:1045500044D81BDFE552E552DF6EDFCFE6FFFC0EED
:10456000DBCFE6FF64EC12F0E552E552E55231D0C4
:104570002BD833D869DFE552E552DF6EFB0EDB50F6
:104580001200DFCFE6FFE66AFC0EDBCFE6FF1AEC97
:104590001EF0E552E552E552E5521BD0DF502B6E7E
:1045A0002C6AFF0ED8802B56000E2C562B50DF6E37
:1045B0001200FE0EDBCFE6FFBFDEE55212002B50ED
:1045C000C808000E2C541200D9CFE6FFE1CFD9FF66
:1045D0001200E552E7CFD9FF1200E652FD0EDBCF05
:0A45E000E6FFFE0EDBCFE6FF12003F
:0645EA00150EE66E010E45
:1045F000E66E0DD8E552E552020173697469150E35
:10460000E66E010EE66E28D8E552E55212001ED97C
:10461000020EE12624D9010E2BC0DBFFFE0EDB507B
:10462000010B05E0010EDBCFE6FFFC0E04D0010E0E
:10463000DBCFE6FFEC0EE66E26EC28F0E552E55205
:104640009F989F9A949C948EAE50DF6EAE50DF6E12
:104650009E9AD9CFE1FFFFD0F9D8E65200D92B506E
:10466000DF6EFE0EDB50010B04E0DFCFE6FFFC0E39
:1046700003D0DFCFE6FFEC0EE66EF4EC27F0E55258
:10468000E552A59AA59898929884E552E4D0DED890
:10469000E65202012E5102E1000E0FD02A512A2BC0
:1046A000EA6A020FE96E070EEA22EFCFDFFF1F0E64
:1046B0002A179D9A2E079D8ADF50E552CCD0020121
:1046C0002E51120002012F511200C0D8E6520201F1
:1046D0002F5102E1000E0FD02B512B2BEA6A220F33
:1046E000E96E070EEA22EFCFDFFF3F0E2B17A39AEA
:1046F0002F07A38ADF50E552AED0A8D8400E0201A2
:10470000385DFCE29D983651362BEA6A620FE96EFD
:10471000070EEA22FE0EDBCFEFFF3F0E3617382BD7
:104720009D8899D093D8100E0201395DFCE2A398C0
:104730003751372BEA6AA20FE96E070EEA22FE0E06
:10474000DBCFEFFF0F0E3717392BA38884D0200E55
:1047500002012E5D13E22C512C2BEA6A020FE96E46
:10476000070EEA22AECFEFFF1F0E2C172E2BABA2A7
:1047700003D0AB98AB88302BABB4322B120066D889
:10478000FD0EDBCF3AF2FE0EDBCF3BF264D002012E
:104790003A513B1101E1000C010C58D8E6526E5021
:1047A000DF6E02013A513B110BE0DFCFE6FF05D08F
:1047B0003BC2FAFF02013A51F96EFADFE5520FD01F
:1047C000400E2F5D0CE22D512D2BEA6A220FE96E6F
:1047D000070EEA22DFCFEFFF3F0E2D172F2B6BA224
:1047E00004D06B986B880201312B6BA402D00201BC
:1047F000332BE55230D00201385102E19D9812006E
:104800003451342BEA6A620FE96E070EEA22EF5048
:10481000AD6E3F0E3417380712000201395102E124
:10482000A39812003551352BEA6AA20FE96E070EE4
:10483000EA22EF506D6E0F0E35173907120006D8B9
:10484000FE0EDBCFE6FF59DFE55205D0D9CFE6FFFC
:10485000E1CFD9FF1200E552E7CFD9FF1200FF0EDA
:10486000E76EFD0EDBCF2BF0E7502B162C6A120003
:104870009EA8FED71200CDD8FE0EDBCFE6FF65EC7A
:104880001AF0E552B9D0C5D80101E150FD0F506FC3
:10489000FF0EDA20516F010EEA6A5025E96E515180
:1048A000EA22B1D850C1E9FF51C1EAFFACD8A4D087
:1048B000B0D8FD0EDBCF2BF0FE0EDBCF2CF02D6A37
:1048C0002BC0E6FF2CC0E6FF2DC0E6FF000EE66E13
:1048D000010EE66E24EC26F0F56E050EE15EF55055
:1048E000000EE66E010EE66E3DEC26F0E552E55256
:1048F000F3CF54F1F4CF55F10101F43408E25451EF
:104900005008000E555503E2500E546F556B566B10
:10491000576B57515519E8AE02D0553504D0545154
:10492000565D555157590EE2000E5625E96E010E9F
:104930005721EA6EEF50AD6E9BDF0101562B000E42
:104940005723E7D7E552E7CFD9FF120062D801011C
:10495000526B1A0E525D0DE2FD0EDBCFE9FFDB2A32
:10496000FE0EDBCFEAFF01E3DB2A4DD80101522B1B
:10497000F0D742D00101C30E506F010E516F0101FB
:10498000C3510201656F666B6751651902E1685199
:10499000661916E00101E3B50ED067C2E6FF65ECCB
:1049A0001AF0E55265C2E6FF65EC1AF0E5520D0E0D
:1049B000AD6E5EDF0101E39565C267F266C268F223
:1049C0000201672B000E6823683507E26751FF0874
:1049D000000E685502E2676B686B1200150EE66EFA
:1049E0003C0EE66E26EC28F0E552E552320EE66EFD
:1049F00091EC29F0E55212000D0EAD6E39DFE55253
:104A0000E7CFD9FF1200EF50E66E65EC1AF0E552E1
:0C4A10001200D9CFE6FFE1CFD9FF120061
:044A1C00D9CFE6FF09
:104A2000E1CFD9FF060EE126100EE66E5FEC13F023
:104A3000E552F3CFDEFFF4CFDDFF0F0EE66E5FEC45
:104A400013F0E552020EF3CFDBFF030EF4CFDBFFD2
:104A50000E0EE66E5FEC13F0E552040EF3CFDBFFB3
:104A6000050EF4CFDBFFDECFE6FFDDCFE6FFC70E9E
:104A7000E66E3F0EE66E89EC28F0E552E552E5520F
:104A8000E552020EDBCFE6FF030EDBCFE6FFBC0EE6
:104A9000E66E3F0EE66E89EC28F0E552E552E552EF
:104AA000E552040EDBCFE6FF050EDBCFE6FFB20ECC
:104AB000E66E3F0EE66E89EC28F0E552E552E552CF
:104AC000E552E80EE66E030EE66EE66AE66AFAEC7A
:104AD0000CF0E552E552E552E552DECF2BF0DDCF8A
:104AE0002CF02C3419E22B508408030E2C5414E2C1
:104AF0007F0EE66EE66A020EE66E7AEC1EF0E55276
:104B0000E552E552000EE66EE66A010EE66E7AECBC
:104B10001EF0E552E552E552020EDBCF2BF0030EFC
:104B2000DBCF2CF02C3419E22B508408030E2C54CC
:104B300014E2000EE66EE66A020EE66E7AEC1EF0F5
:104B4000E552E552E552FF0EE66EE66A010EE66EAC
:104B50007AEC1EF0E552E552E552040EDBCF2BF065
:104B6000050EDBCF2CF02C3419E22B508408030EF9
:104B70002C5414E2FF0EE66EE66A020EE66E7AEC44
:104B80001EF0E552E552E5527F0EE66EE66A010E32
:104B9000E66E7AEC1EF0E552E552E552D9CFE1FF20
:084BA000E552E7CFD9FF120036
:084BA8001E0EF66E080EF76EFA
:104BB000000EF86E02010900F550466F0900F5502D
:104BC000476F03E1466701D03DD00900F550416FC2
:104BD0000900F550426F0900F550436F09000900C4
:104BE000F550E96E0900F550EA6E09000900090068
:104BF000F550446F0900F550456F09000900F6CFE4
:104C000048F2F7CF49F2F8CF4AF241C2F6FF42C26A
:104C1000F7FF43C2F8FF0201445302E1455307E0A6
:104C20000900F550EE6E4407F8E24507F9D748C28F
:104C3000F6FF49C2F7FF4AC2F8FF02014607000E1D
:084C4000475BBFD71200120010
:084C4800FB0EE3CFF6FFFC0EAA
:104C5000E3CFF7FFFD0EE3CFF8FFFE0EE3CFE9FF52
:104C6000FF0EE3CFEAFFE9CFF3FFEACFF4FF09003D
:104C7000F5CFEFFFEE66FBD71200FE0EE3CFE9FFA4
:104C8000FF0EE3CFEAFFF36AF46AEE5203E0F34A61
:104C9000F42AFBD71200FF0EE3CFF8FFE552FF0E18
:104CA000E3CFF7FFE552FF0EE3CFF6FFE552E66AEA
:104CB000E66AE66A0900F55209E0FD0EE32A05E11D
:104CC000FE0EE32A02E1FF0EE32AF4D7FD0EE3CF46
:104CD0001CF0FE0EE3CF1DF0FF0EE3CF1EF012001E
:104CE0001DC029F01D502202F4CF1CF0F3CF1BF0A1
:104CF0001E502302F4CF1EF0F3CF1DF02202F3501A
:104D00001C26F4501D22E86A1E2229502302F3506B
:104D10001C26F4501D22E86A1E22000C1EC02AF038
:104D20001DC029F01D502202F4CF1CF0F3CF1BF060
:104D30001E502302F4CF1EF0F3CF1DF02202F350D9
:104D40001C26F4501D22E86A1E2229502302F3502B
:104D50001C26F4501D22E86A1E2223AEB4EF26F072
:104D600029501D5E2A501E5A2AAE000C22501D5E8C
:064D700023501E5A000C46
:0A4D7600D9CFE6FFDACFE6FFE1CF68
:104D8000D9FFE2CFDAFFE652E652E652E652D950B8
:104D9000FB0F2B6EFF0EDA202C6E2BC0DEFFDD6EBC
:104DA000DECFE6FFDDCFE6FFFB0EDBCFE6FFFC0E3E
:104DB000DBCFE6FFFD0EDBCFE6FF73C2E6FF74C27A
:104DC000E6FF50EC04F0F56E070EE15C02E2E16AEA
:104DD000E552E16EF550020EF3CFDBFF030EF4CF88
:104DE000DBFF020EDBCF2BF0030EDBCF2CF02BC052
:104DF000F3FF2CC0F4FFD9CFE1FFDACFE2FFE55299
:0A4E0000E5CFDAFFE7CFD9FF12007B
:064E0A00D9CFE6FFDACF6C
:104E1000E6FFE1CFD9FFE2CFDAFFFB0EDBCF2BF0CD
:104E2000FC0EDBCF2CF00001800E2C141AE1FB0EDF
:104E3000DBCFE9FFFC0EDBCFEAFFEECFF3FFEDCFD8
:104E4000F4FFEE2A000EEF22F3CFE9FFF4CFEAFFE2
:104E5000FD0EDBCFEFFFEF502C6AF36E2CC0F4FF9A
:104E600010D0FB0EDB50FE0806E1FD0EDBCFE6FFA7
:104E7000A1EC29F005D0FD0EDBCFE6FF1FEC24F0FE
:0E4E8000E552E552E5CFDAFFE7CFD9FF120089
:024E8E0002011F
:104E9000010E6F6F706BE85070110AE0FF0EE66E46
:104EA000E66A030EE66E7BEC1EF0E552E552E55233
:104EB0000201020E6F6F706BE850701129E0000E56
:104EC000E66EE66A030EE66E7BEC1EF0E552E552F6
:104ED000E5526FC22BF070C22CF02D6A2E6A2CAEF8
:104EE00002D02D682E682BC0E6FF2CC0E6FF2DC037
:104EF000E6FF2EC0E6FF010EE66E37EC0DF0F56E14
:104F0000050EE15EF550010EE66E2CEC0DF0E5525B
:024F100012008D
:0E4F12001B502002F3CF17F0F4CF18F021024D
:104F2000F3501826000EF420196E1B502202F35085
:104F30001926000EF4201A6E1B502302F3501A2675
:104F40001C502002F3501826F4501922000E1A2289
:104F50001C502102F3501926F4501A221C50220230
:104F6000F3501A261D502002F3501926F4501A222D
:104F70001D502102F3501A261E502002F3501A260B
:024F800012001D
:0E4F8200D9CFE6FFDACFE6FFE1CFD9FFE2CFCD
:104F9000DAFF3F0EC716C66AFD0EDB50C612FB0EC7
:104FA000DB50C712FC0EDB50030A09E0010A04E0E3
:104FB000020A06E1C78C04D0C78CC68801D0C68817
:104FC000FD0EDB50050A03E0010A04E1928A948693
:104FD000C79E01D09496949A9488C68AE552E5CFEC
:084FE000DAFFE7CFD9FF120050
:084FE800D9CFE6FFDACFE6FFA6
:104FF000E1CFD9FFE2CFDAFF6C6A6B6AFD0EDBB05E
:105000006C88DBA202D06C8C6B8CDBB46C8EDBA664
:1050100002D06B8801D06B8ADBA802D06C8401D0EF
:105020006C94DBAC02D0A38A01D0A39ADBAE02D091
:10503000A38801D0A398FC0EDB506F6E6C8A6B8E38
:0C504000E552E5CFDAFFE7CFD9FF120000
:04504C00D9CFE6FFD3
:10505000DACFE6FFE1CFD9FFE2CFDAFFAC6AAB6A85
:10506000FD0EDBB0AC88DBA202D0AC8CAB8CDBB429
:10507000AC8EDBA602D0AB8801D0AB8ADBA802D015
:10508000AC8401D0AC94DBAC02D09D8A01D09D9A57
:10509000DBAE02D09D8801D09D98FC0EDB50AF6E38
:1050A000AC8AAB8EE552E5CFDAFFE7CFD9FF12002D
:1050B000D9CFE6FFDACFE6FFE1CFD9FFE2CFDAFFC3
:1050C000C26AC16AC06AFC0EDB407F0B3C0BC26E39
:1050D000FD0EDB500F0B2B6EFC0EDB38F00B300B94
:1050E0002B10C16EFD0EDB380F0B070B2B6EFD0E68
:1050F000DB50800B2B10C06EFC0EDBAE03D09E9CF1
:105100009D8CF28CC280E552E5CFDAFFE7CFD9FF64
:0251100012008B
:0E511200D9CFE6FFE1CFD9FF020EE126D9503A
:10512000FD0F2B6EFF0EDA202BC0DEFFDD6EDECF13
:10513000E6FFDDCFE6FFFD0EDBCF2BF0FE0EDBCF73
:105140002CF02D6A2BC0E6FF2CC0E6FF2DC0E6FF39
:1051500073C2E6FF74C2E6FF50EC04F0F56E070E72
:10516000E15EF550D9CFE1FFE552E7CFD9FF12005C
:10517000D00EE66E070EE66EE66AE66AFAEC0CF012
:10518000E552E552E552E5527F0EE66EE66A080EFC
:10519000E66E7AEC1EF0E552E552E5527F0EE66EC1
:1051A000E66A020EE66E7AEC1EF0E552E552E55232
:1051B0007F0EE66EE66A010EE66E7AEC1EF0E552B0
:0A51C000E552E5520EEC25F0FDD794
:0651CA001A6A196A186A56
:1051D000176A200EE76ED8901B361C361D361E3619
:1051E0001736183619361A362050175C21501858C1
:1051F0002250195823501A5809E32050175E2150A5
:10520000185A2250195A23501A5A1B2AE72EE4D74B
:0252100012008A
:0E521200D9CFE6FFDACFE6FFE1CFD9FFE2CF3A
:10522000DAFFFD0EDB507E0BCD6EFD0EDBAC02D047
:10523000CD8E01D0CD9ECF6ACE6A9E90DBAE02D0DD
:105240009D8001D09D90CD80E552E5CFDAFFE7CF7C
:04525000D9FF120070
:0C525400E66AE66A7EEC1CF0E552E552CA
:10526000010EE66EE66EE66EE66EE66EE66EE66EE3
:10527000E66EE66EE66EE66EE66EE66EE66EE66E8E
:10528000E66E100EE66ECCEC11F0F56E110EE15EDE
:04529000F5501200C3
:0C529400D9CFE6FFDACFE6FFE1CFD9FF6B
:1052A000E2CFDAFFE652E652C350DF6E010EC4CF02
:1052B000DBFFDECF2BF0DDCF2CF02BC0F3FF2CC0BB
:1052C000F4FFE552E552E552E5CFDAFFE7CFD9FF2B
:0252D0001200CA
:0E52D2001A6A196A100EE76ED8901D361E3645
:1052E00019361A362250195C23501A5805E32250F9
:0E52F000195E23501A5A1D2AE72EF0D712001D
:0252FE00F36A51
:10530000F46AFF0EE124E96EFF0EE220EA6EED661C
:1053100007D02F0EEF6404D03A0EEF6001D0F32ACD
:02532000120079
:0E532200FF0EE350366E480E01D04C0EE76EC3
:10533000E72EFED7E76AE72EFED7362EF7D7000016
:02534000120059
:0E534200FF0EE350ACBA04D0AF6AAB8EAC8A5B
:0E535000949CACA2FED7AD6EF36EF46A120010
:02535E00FF0E40
:10536000E350E84E1200000000D000D000D0E82E3C
:04537000FAD7120056
:0C5374003031323334353637383961625D
:05538000636465660096
:0B53850000878F979FA7AFB7BFC7CF6F
:06539000D7DFE7EFF7FF95
:0A539600D9CFE6FFE552E7CFD9FFBB
:0253A0001200F9
:0C53A200D9CFE6FFE552E7CFD9FF12009B
:0253AE00C290AB
:0453B0009D9C1200AE
:0453B400C28212009F
:0253B800FEFFF6
:0653BA00000000000000ED
:0C53C000000000000000000000000000E1
:0453CC0000000000DD
:0953D0000000000000000000FFD5
:0453D90000000000D0
:0353DD00000000CD
:1053E00000000000000000000000000000000000BD
:1053F00000000000000000000000000000000000AD
:10540000000000000000000000000000000000009C
:0954100000000000000000000093
:0354190000000090
:04541C000000001478
:01542000008B
:020000040030CA
:0E000000FFFEFEFCFFFEFBFFFFFFFFFFFFFF0A
:00000001FF
